:1000000012C02BC029C028C004C126C025C024C0EE
:1000100023C022C021C020C01FC029C01DC01CC0D9
:100020001BC01AC019C011241FBECFEDCDBF10E0F8
:10003000A0E6B0E0E8E4F3E002C005900D92AE3631
:10004000B107D9F710E0AEE6B0E001C01D92A437C9
:10005000B107E1F720D176C1D3CF1F920F920FB62F
:100060000F9211240F900FBE0F901F9018951F92A2
:100070000F920FB60F9211242F933F936F937F939C
:100080008F939F93EF93FF9382991AC08091720090
:1000900090917300019690937300809372008FEF9C
:1000A00094E090936C0080936B00809171008823A2
:1000B00021F082E08093710019C01092710016C087
:1000C00080917200909173008134910558F0809175
:1000D0006E008F5F80936E008FEF98E090936C00BE
:1000E00080936B00109273001092720080917200E6
:1000F000909173008F5F924099F410927300109268
:10010000720080916E008F5F80936E0080916E0010
:10011000833618F082E0809371008BE380936F0048
:100120008091700090E289278093700080916B002D
:1001300090916C00892B09F45AC080916B009091CA
:100140006C00019790936C0080936B00809171001C
:100150008130B9F480917100833011F435E601C02B
:1001600030E080916B0090916C0084709170892BCD
:1001700021F080917000846001C084E082BB8FED2B
:1001800015C080917100823021F48FEF88BB30E080
:100190000EC084E082BB80916E00882321F03091F4
:1001A0006E003F5F02C030916F008FEF88BB80917F
:1001B0007000882371F428B3832F6AE0B7D0E92F49
:1001C000F0E0E05AFF4F80818095822388BB909AAF
:1001D00013C028B3832F6AE0A9D0E82FF0E0E05ADB
:1001E000FF4F80818095822388BB919A05C018BA01
:1001F00084E082BB80E489BFFF91EF919F918F9152
:100200007F916F913F912F910F900FBE0F901F9094
:1002100018951F920F920FB60F9211242F938F9360
:100220009F9380916F00882321F080916F0081500F
:1002300019C080917100882321F082E080937100C1
:1002400013C08BE380936F0080916E00882331F0A0
:1002500080916E00815080936E0006C081E0809393
:1002600071008EE080936F0080916B0090916C0024
:100270008F5F964030F48FEF96E090936C00809300
:100280006B0081E489BF9F918F912F910F900FBEDA
:100290000F901F90189522E020936F0081B5886120
:1002A00081BD11BC83E281BB8FEF87BB80E888B939
:1002B00088E09DE39BBD8ABD1FBC8CE08EBD80E5C0
:1002C00086BF20BF23BF80E489BF25BF789424E682
:1002D00030E0A0E474E060E35BE340E28091710011
:1002E0008230D9F480ED97E0F9013197F1F7019769
:1002F000D9F7829BFECF80ED97E0F9013197F1F7B6
:100300000197D9F7ABBF72BB65BF88951BBE5093F1
:100310006F0010926E001092710080916B009091AE
:100320006C00892BD9F645BF8895D8CF991B79E009
:1003300004C0991F961708F0961B881F7A95C9F775
:0803400080950895F894FFCFA9
:0E034800CF035D5B93DADE43DFDB9EFF040034
:00000001FF
